:100000000C94C2170C94EA170C94EA170C94EA1794
:100010000C94EA170C94EA170C94EA170C94EA175C
:100020000C94EA170C94EA170C94DE190C94501AED
:100030000C94EA170C94EA170C94EA170C94EA173C
:100040000C94EA170C949C1E0C94EA170C94EA1773
:100050000C94EA170C94EA170C94EA170C94641D9C
:100060000C94EA170C94EA170C94EA170C94EA170C
:100070000C94EA170C94EA170C94EA170C94EA17FC
:100080000C94AE1D0C94EA170C94EA170C94EA1722
:100090000C94EA170C94EA170C94EA170C94EA17DC
:1000A0000C94EA170C94EA170C94EA17F0F89C8E5B
:1000B0008783878E9CF8F00000FEFF030303030391
:1000C000070EFCF80000FEFF0303030303070EFC0A
:1000D000F80000FFFF00000000000000FFFF00002C
:1000E000FEFF8383838383C7EE7C380000F8FC0E19
:1000F00007030303070EFCF800003F7FE0C0808089
:10010000C0E07F3FFFFF01010101010101FFFF008E
:1001100000FFFF0C0C0C0C1C3E77E3C100007FFFBE
:10012000C0C0C0C0C0E0703F1F00001F3F70E0C0F3
:10013000C0C0E0703F1F00007FFFC1C1C1C1C1E36B
:10014000773E1C00001F3F70E0C0C0C0E0703F1F42
:10015000000000000001FFFF01000000D5F08D1439
:10016000A1C881CFD9F1AF200054494521007CFCC2
:10017000F8C080E0E0E000E0F8FC380000FCFCFCA7
:100180000000FCFCFCF0E0C0FCFCFC0000FCFCFC03
:10019000F0E0C0FCFCFC00FCFCFCDCDC9C1C00FC7B
:1001A000FCFC9C9CFCF8F00000FEFEFE00010F1F12
:1001B0001F0F030F1F1F07010000001F1F1F00005C
:1001C0001F1F1F0103071F1F0F00001F1F1F010319
:1001D000071F1F0F001F1F1F1D1D1C1C001F1F1F9F
:1001E000070F1F1F0D000073777300000000C03061
:1001F00008048444A2A2A2B2545458D060800000E3
:100200000000000000000000000000003C67E42C3B
:100210001E3BCE971C2227221015DFD11D061EE0A3
:10022000000000000000000000000000FF386080B7
:100230000080434F7F58F0B03030B0E87C46F31C6C
:1002400008F8000000000000000000030708111F6C
:1002500038D0101010180F01C33D60C080E0F3FDCE
:10026000FDFC7C1800000000000000000000003CC5
:100270007B787C7E3E3F1F1F0F07010303030101B4
:100280000000000000000000E038CCF6FA7ABB5D08
:100290005D5D4DABAAA62C9870C000000000000068
:1002A0000000000000007EC3981BD3E1C43168E366
:1002B000DDD8DDEFEA202EE2F9E11FF000000000BA
:1002C000000000000000FF00C79F7FFF7FBCB080E0
:1002D000A70F4FCFCF4F1783B90CE3F604FC0000F4
:1002E0000000000000070C18372E60C72FEFEFEF5B
:1002F000E7F0FE3CC29F3F7F1F0C02020382E63CF8
:100300000000000000000000007EC384878381C1DC
:1003100040602030180E04040406020301000000AF
:100320000000000080404080C0C0C0C0C0C040404D
:1003300040404040404040C0C080000000000000FD
:100340000000000F10102325454DCD1D0E02004565
:100350009265E0D4E0957F120E03000000000000DB
:10036000000000000000E01008FF00808000000096
:10037000E19D0301000000000000000000000000FB
:1003800000000000000001020304040831C71A64E1
:1003900038A39C90F0504848700000000000000016
:1003A0000000000000000000000000000302010146
:1003B0000101000000000000000000000000C0601B
:1003C000A0A060202020202020A0A0A0A0A0A0A06D
:1003D000A0A0202060C0800000000000001F302F7F
:1003E0006F5CDABAB232E2F1FDFFBA6D9A1F2B1FD1
:1003F0006A80ED311C0700000000000000000000D2
:10040000F018ECF700FF7F7FFFFFFF1E62FC860302
:1004100001000000000000000000000000000001DA
:100420000306050C0B1B77CE38E59BC75C636E0893
:10043000ACB4B48CF8000000000000000000000024
:10044000000000000000070405060202020301018B
:10045000000000000000000000000000000000009C
:1004600000000000808000008040C000000000000C
:10047000000000000000000000000000000000F884
:10048000948203F0095999481063ADF3000000000D
:100490000000000000000000000000007884BFE0C1
:1004A000041F0B1021242D2CE55E433F00000000AB
:1004B0000000000000000000000000E020603F0A93
:1004C0008ACA526262528A979888780000000000B7
:1004D0000000000000000000000001010101010116
:1004E000000000000000000000000000000000000C
:1004F0000000000000000000000000000080C0407C
:1005000040C0C060A020E08080000000000000002B
:10051000000000000000000000FC066B7DFC0FF6F0
:10052000A666B7EF9C520CFF8000000000000000A0
:10053000000000000000FC867B401FFBE0F4EFDEC3
:10054000DBD2D31AA1BCC07F000000000000000075
:100550000000000000F011D19FC0F57535AD9D9DE4
:10056000AD7568677484FC000000000000000000A6
:100570000000000003020202020202030100000167
:100580000101010101000000000000000000000066
:10059000000080800080808080000000804020403B
:1005A00020E000000000000000000000F0484C9631
:1005B000234C9021C618E0437F7F6182C73AC8C8A8
:1005C0004ACF90E000000000000000C1271E140D7B
:1005D0000A0407060508800000100F110A150D1FF8
:1005E000FF040808101020C00000070808080404D1
:1005F000040202020509183868C888183C64C382DE
:1006000004040408080807000000000000000000BF
:1006100000000000000000000103030100010303CB
:10062000010000000000000000000080C04040C049
:1006300040404040C080C060B0D0B0D010F08000DA
:10064000000000000000F80CB6B369DCB36FDE39BF
:10065000E71FBC80809E7D38C53737B5306F18F0F6
:100660000000000000E33ED8E1EBF2F5FBF8F9FAF8
:10067000F77FFFFFEFF0EEF5EAF2E000FBF7F5ECB5
:10068000E8D830E00F181717171B0B0B0D050D1AC4
:100690003667C7973777E7C39B3C6DCB8B9B1717A4
:1006A00017180F000000000000000000000000000C
:1006B0000000030604040603060404060300000009
:1006C00000000000000000F0086848100828A82872
:1006D000A4220422A428E8F8700000000000000012
:1006E0000000000000C03C67C3408074880A31727B
:1006F000F4F2D2F63D12C8791E000000000000009E
:100700000000001FF0C00000000D314243830202D0
:100710000202027F41FBACA8F800000000000000CC
:1007200000000000030F1C34E8352B140F0101C337
:100730003D60C08020139DF5EC741800000000009F
:100740000000000000003C6340646222351B1D0F66
:100750000701030303010100000000000000000086
:1007600000F80CF494B4ECF4D454D65BDDFBDD5B00
:10077000D614048CF800000000000000000080E0A7
:100780003FC3983CBF7F8B77F5CE8D0B0D2D09C2F3
:10079000ED3786E13F00000000000000003FE00F61
:1007A0003FFFFFFFF2CEBDBC7CFDFDFDFDFD80BE29
:1007B00004535604FC000000000000000001071C68
:1007C0003063CB17CAD4EBF0FEFE3CC29F3F7FDF05
:1007D000EC620A138AE63C00000000000000000002
:1007E0007EC39CBF9B9DDD4A642230180E04040426
:1007F00006020301000000000000000000000000ED
:1008000000000000000000000000000000000000E8
:10081000000000000000000000E0306828A8D03090
:100820007070E0E0E6F9A97FE018846428485090F1
:10083000A0EEFEFC000000000F1427C44549BC4F89
:100840005727232321F1111F807F000000000000A3
:100850000101010000000000000E090A0B3A7EF9B8
:10086000F9DEEAE965040203000000000000000070
:100870000000000000000000000000000000000078
:100880000000000000000000000000000000000068
:100890000000000000000000000000000000000058
:1008A00080808080800000000000000000000000C8
:1008B000000000F018CC94D4542CC88888181F1954
:1008C0000656801FE67A9AD6B4AC685F110103FE23
:1008D00000001F306BD83BBAB643B0A8D8DCDCDED2
:1008E0000EEEE07F80FF0000010103020202030020
:1008F0000000001F11161574C58106062115169AF1
:10090000FB0D0407000000000000000000000000D4
:1009100000000000000000000101010101010100D0
:1009200000000000000000000000000000000000C7
:1009300000000000000000000000C02010C8248457
:10094000444444444848505060C000000000000047
:10095000008040202030101E1113121F7E8B123F8A
:1009600041858555CD819DF5FF0000000000000FF9
:10097000101E21A1E1D1CE80808000000081828400
:100980009890101090F844433E00000000000000D2
:100990000000070811E1C30303030303079C640479
:1009A000070303874830000000000000000000003B
:1009B000000000071F3C787878783E3D7C7C7C7C8A
:1009C0003E010000000000000000000000000000E8
:1009D0000000000000000000000000000000000017
:1009E0000000000000000000000000000000000007
:1009F000000080E030D8EC36DA7ABABABABAB6B4C7
:100A0000ACA89830E00000000080C060B0D0D8C82A
:100A1000EFE1EEECEDE08174EDC0BE7A7AAA327EB1
:100A2000620A00FF000000001F302F61DE5E1E2EF4
:100A3000317F7F7FFFFFFF7E7D7B676FEFEF6F076B
:100A4000BBBCC17F000000000000000F18B7EE1E05
:100A50003CFCFCFCFCFCF8639BFBF8FCFC78B7CD91
:100A60007800000000000000000000000F3860C3A4
:100A700087878787C1C283838383C17E0301000088
:100A80000000000000000000000000000000000066
:100A90000000000000000000000000000000000056
:100AA0000000000000000000000000000000F80648
:100AB000FAFCF8FE02FCF800000000000000000054
:100AC0000000000000000000008080804040433CA7
:100AD0000901054D849159954EFC0000000000006D
:100AE0000000007C82827129A8740C0000000000C4
:100AF00000010204C5350D0A097182827C000000E4
:100B0000000000000304083FC00000F81028C000E7
:100B100018E40300000000000000000000000000D6
:100B20000000000000000C33C01E23C00C33C01EA8
:100B300023C00000000000000000000000000000D2
:100B400000000000000000000101010000000101A0
:100B50000100000000000000000000000000000094
:100B600000000000000000FC07F905030701FD0379
:100B700006FC808000000000000000000000000073
:100B80008080C0404060A1A7BCC3F6FEFAB27B6E75
:100B9000A66AB103FE80000000000000FE837D7D98
:100BA0008ED6578BF3FFFFFFFFFFFFFEFDFB3ACA18
:100BB0007215F68E7D7D83FE0000000001070C1B80
:100BC00077C03FFFFF07EFD73FFFE71BFC070100A0
:100BD0000000010101010000000000000000001EF3
:100BE00073CC3FE1DC3FF3CC3FE1DC37E0000000B9
:100BF00000000000000000000000000000000000F5
:100C000001030202020301030202020300000000CA
:100C100000000000000000000000000000000000D4
:100C200000000000808000008040C0000000000044
:100C3000000000000000000000000000000000F8BC
:100C400014020330C91999D810A3ED130000000055
:100C5000000000000000000000003048CCD2CA4B69
:100C60000C0E0910202529E8615F5048483000002B
:100C70000000000000000000000000C0407F0A0AE1
:100C80000A12E222120A8F48300000000000000021
:100C900000000000000000000000030408080A0F24
:100CA000010102040405070000000000000000002C
:100CB0000000000000000000000000000000000034
:100CC0000000000000000000000000000000000024
:100CD00000000000000000000000000080C0404054
:100CE000C0C060A020E08080000000000000000084
:100CF0000000000000000000FC06EBFDFCCF36E623
:100D00006627EF5C12EC3F000000000000000000CE
:100D100000000078CCB6332D35B4F3F1F6EFDFDA0E
:100D2000D6179EA0AFB4B4CC78000000000000003D
:100D300000000000E121BF80F5F5F5ED1DDDEDF5CA
:100D400070B7CC7800000000000000000000000038
:100D5000000000070C1B171715101E060D0B0B0AC1
:100D6000080F00000000000000000000000000006C
:100D70000000000000000000000000000000000073
:100D80000000000000000000000000000000000063
:100D9000000000000000000000008040204020E033
:100DA00000000000000000000000000080C0609013
:100DB0001020D0101070E03E6186093E4C48CCCF28
:100DC00090E0000000000000003EE9C99264493252
:100DD00024382B44020302130F100810081FFF3E93
:100DE00040408080000000003E41404020202030F4
:100DF000305068CCC0C0404040C0E02018172020D0
:100E0000204040413E0000000000000000000000C3
:100E100000081F1F0800081F1F0800000000000036
:100E200000000000000000000000000000000000C2
:100E300000000000000000000000000000000000B2
:100E400000000000000000000000000000000000A2
:100E5000000080C060B0D0B0D010F0800000000072
:100E60000000000080C060309868E8D828E8E88872
:100E70001FC19E79F6C1B3B733306F18F000000080
:100E800000007FC116366D9BB6CDDBC7D4BBFDFC21
:100E9000FDECF0EFF7EFF7E000C1BFA16040C080CC
:100EA000007FC1BEBFBFDF5F5F4FCFAF97333F3F14
:100EB000BFBFBF3F1FDF67685F5FDFBFBFBEC17FD0
:100EC000000000000000000000001C372020371D3B
:100ED000372020371D000000000000000000000047
:100EE0000000000000000000000000000000000002
:100EF00000000000000000000000000000000000F2
:100F00000000000000000000F00868481008C888D1
:100F100088840204028488C8F87000000000000081
:100F200000804020A0B0901C67C3408074880B12E2
:100F300013147252771E13C8791E00000000000FB0
:100F4000101E212A2AAAFF0906000101020303023A
:100F50000202020281FFAAAA7C0000000000000039
:100F6000000000000F90E14000000000009C6000C5
:100F70000000028748300000000000000000000070
:100F8000000000071820704072423E2170427242F9
:100F90003E01000000000000000000000000000012
:100FA0000000000000000000000000000000000041
:100FB0000000000000000000000000000000000031
:100FC00000F80CF494B4ECF43474767BFDFBFD7BF8
:100FD0007634048CF80000000080C060B0D058481F
:100FE0006FE3983CBF7F8B77F4EDECEB8DAD88E140
:100FF000EC3786E13F0000001F302F615E55D5556C
:1010000000F6F9FFFEFEFDFCFCFDFDFDFDFD7E0092
:10101000555583FE0000000000000000009FF06FA7
:101020001EBFFFFFFFFFFF639FFFFFFFFD78B7CDF0
:101030007901000000000000000000000F3867DFA9
:101040008FBF8DBDC1DE8FBD8DBDC17E0301000090
:101050000000000000000000000000000000000090
:101060000000000000000000000000000000000080
:10107000000000000000000000000000000000FE72
:10108000FE82FE82FE82FE000000000000000000E2
:1010900000000000000000E02020C000768E87C61F
:1010A000B70E174677FF8EF620E000000000000024
:1010B0000000000000003F212F14120938C403076C
:1010C0001F7F7CBF7F1337211F000000000000003E
:1010D0000000000000000000000000007F8101FF10
:1010E0008301FF000000000000000000000000007D
:1010F00000000000000000000000001C3FF0FFEFB7
:10110000C83FF87000000000000000000000000070
:1011100000000000000000000000000000010101CC
:1011200000000000000000000000000000000000BF
:101130000000000000000000FF01017D017D017D35
:1011400001FF00000000000000000000000000009F
:10115000F010D0D030FF8971783948F1E8B98800B3
:101160007109DF10F0000000000000000000007FA7
:10117000405E506B2D76C73BFCF8E080834080ECEE
:10118000485E603F0000000000000000000000001A
:101190000000000000FF807EFE007CFE00FF0000DB
:1011A000000000000000000000000000000000003F
:1011B000000000003E63C00F001037C0078CF8002D
:1011C000000000000000000000000000000000001F
:1011D0000000000000010302020203010100000000
:1011E000000000000000000000000000000000807F
:1011F00040201010101010101010906020C000003F
:1012000000000000000000000000000000000000DE
:10121000000080407E4180804060504840605876A9
:1012200049544B5F704040404040E0206020202007
:10123000C00000000018244243E41C040300000026
:10124000000000002010F84848380808080808087E
:101250000F10101010100F000080C0402018060161
:10126000038343432333CB47070707068F700000F0
:101270000000000000000000000000000000001F4F
:101280001F1818181C0201000000060D0E0E0E0E8D
:101290000E0F0F0C00000000000000000000000016
:1012A000000000000000000000000000C060B0D896
:1012B000E8E8E8E8E8E8E8E86898D030E00000000E
:1012C000000000000000000000000000000000C05E
:1012D00060BF81BE7F7FBF9FAFB7BF9FA789B6ABFF
:1012E000B4A08FB8A0A0A0B010D090D0D0D030E0E3
:1012F00000003C66DBBDBC1BE3FBFCFFFFFFFFFF08
:10130000FFFFDFEF07B7B7C7771717171717302F8C
:101310002F2F2F2F301FC06020B0DCE7F9FEFC7CA0
:10132000BCBCDCCC34B8F8F8F8F9708FF8000000D9
:101330000000000000000000000000003F20202707
:101340002727233D0603010F191211111111111046
:1013500010131E000000000000000000000000004C
:10136000000000000000000000000000808080807D
:101370008080C0C0C0C0C0C0C0C0C0C0800000006D
:10138000000000000000000000000000000000005D
:101390000000010302050505C5251E0620222622A0
:1013A000282C2A273E20202020202020C0000000BA
:1013B000000000000000000080402020E01807002E
:1013C0000000010181635B4727190101010102024D
:1013D0000202010000000000000080808080434481
:1013E00028988740300818A4400699600000000043
:1013F00000000000000000000000000000000000ED
:1014000001060812161713121C00000709080A0B20
:101410000A0A09090E000000000000000000000098
:10142000000000000000000000C04040404040605C
:101430002020202020202020202060C080000000CC
:101440000000000000000000000000000000000399
:1014500006040D0A0AEA3ADAE1F9DFDDD9DDD7D36D
:10146000D5D8C1DFD0D0D0D0D0D030E0000000003F
:101470000000000000C060B0D0D01CE7F8FFFFFF04
:10148000FEFE7E9CA4B8D8663E0202060505050550
:1014900006030000000000C040404067ACBBD767B7
:1014A00078BFCFF7E75BBFF9669FF0808000000050
:1014B00000000000000000000000000000030E1902
:1014C000372D292A2C2D233F0F1816171514151503
:1014D0001616111F000000000000000000000000B0
:1014E00000000000000000000000000000000000FC
:1014F00000000000804020300898909088043CD084
:10150000300000000000000000000008100800C0CB
:10151000C086CF1E0F8660AE31314941627C930C8C
:1015200001D9DDC11AFE414080000000000000002A
:1015300000000000000001F1101C0283C244792267
:10154000A46830080809090B090906050202010010
:101550000000000000000000000000000000010288
:10156000020203020404050700000000000000005E
:10157000000000000000000000000000000000006B
:10158000000000000000000000000000000000005B
:10159000000000000000000000000000000000004B
:1015A000000000000000000000808080808000803B
:1015B00080C060B0D8CCF4646C6C76FAC22EC8F8E7
:1015C00000000000000000001C342C34FC202F79A7
:1015D00030E1F0799F51CECEB6BE9D836CF3FE26EE
:1015E000223EE501BEA360C0000000000000000034
:1015F00000000103FA0AEFE3FD7C3DBB86DD5B974B
:10160000CF77171616141616190A0D0506030000D3
:1016100000000000000000000000010306050505B1
:10162000040D0B0B0A080F00000000000000000072
:1016300000000000000000000000000000000000AA
:10164000000000000000000000000000000000009A
:10165000000000000000000000000000000000008A
:10166000000000000000000000000000000000007A
:10167000000000000000000000000000000000006A
:1016800000000000000080C060901020D010107892
:10169000E80808F010109060408000000080008092
:1016A000800000000000000000003EE9C992A4494B
:1016B00092F4080B1422A36203020202ABD48685C3
:1016C000820209147998939C9820C00000000000C1
:1016D0000000010204091A2B2C5868CCC3C04040FA
:1016E00040C0E02018070001010101070F000101BF
:1016F00001000000000000000000000000000000E9
:1017000000020707020002070702000000000000B5
:1017100000000000000000000000000000000000C9
:1017200000000000000000000000000000000000B9
:1017300000000000000000000000000000000000A9
:10174000000080C060309868E8D828E8EC8414F481
:10175000F40CE8E86898B060C080C040C04040C069
:10176000000000000000007FC116366D5BB66D0BF7
:10177000F7F4EBDD5C9DFCFDFDFD542B797A7DFDDE
:10178000F6EB86676C6366DC30E000000000010366
:10179000060D1B366554D3A797333C3FBFBFBF3FF1
:1017A0001FDF67380F0202020E18101F0202020329
:1017B0000000000000000000000000000000070D15
:1017C00008080D070D08080D0700000000000000C4
:1017D0000000000000000000000000F00868481051
:1017E00008C88888840204028488C8F87000000051
:1017F0000000000000000000805C6743C080748827
:101800000B1213147252771E13C8799E40A0A0C009
:101810008000003C424F506535F50F04030203037E
:101820000202020202070DF386CF69371A0A070087
:101830000000000080403E01000000C0301030D8A1
:10184000080404020F70C000000000000000000641
:101850000911141C141C141E0D00000000070C08B4
:101860000A0A0E0A0F0A0C00000000000000000027
:101870000000000000000000000000000000000068
:101880000000000000000000000000000000000058
:1018900000000000000000000000F80CF494B4EC1C
:1018A000F43474767BFDFBFD7B7634048CF8000009
:1018B000000000000000000000000000000080C0E8
:1018C0007FA398BC3F7F8B77F4EDECEB8DAD88E187
:1018D000EC3786A1BFA0A0B090509050505030E09F
:1018E00000007EC3BDB0AF1ACAEAF0FBF8E5FCFC0D
:1018F000FDFDDDED05F61617171717171717171447
:1019000011141515180FC060A0B0DCE7F9FEFF7FB9
:10191000BFBFDFCF37B9FFFFFFFB708FF8000000BC
:101920000000000000000000000000003F202F2702
:101930002F27233D0603010F191215151511151038
:1019400014131E0000000000000000000000000052
:101950000000000000000000000000000000000087
:10196000000000FCFC04FC04FC04FC00000000007F
:101970000000000000000000000000000000000067
:1019800000000000000000EC1C0F8D6F1D2F8DEF7C
:10199000FF1CEC0000000000000000000000000040
:1019A00000000000000000000000000000000779B7
:1019B00089090939F959794D4D7505050505070955
:1019C00009090700000000000000000000008080FE
:1019D00040201088442293924A4E33A284586000DB
:1019E00000000000000000000000000000000000F7
:1019F000001F3F39341C1A010100000307060607C7
:101A000007060600000000000000000000000000C3
:101A100000000000000000000000000000000000C6
:101A2000FE0202FA02FA02FA02FE000000000000C2
:101A300000000000000000000000000000000000A6
:101A400000000000FE12E3F07290E2D0721000E39A
:101A500012FE808080808080808080800000000076
:101A600000000000000000000000010FF88676F67C
:101A7000F6C606A686B2B28AFA0A0A0A1816161618
:101A8000180F000000000000808080C04060B0D8C7
:101A9000EC76BBDD6C6DB5B1CC5D7BA69CF0000037
:101AA00000000000000000000000000000003F6097
:101AB00040464B63253E0203070C08090908080944
:101AC000090F0000000000000000000000000000FE
:101AD000000000000000C02010C824844444444496
:101AE0004848505060C000000000000000000000A6
:101AF00080404E71B3B2AF7E8B123F41858555CD8C
:101B0000819DF5FF402020408000003C424F506006
:101B1000E0D08F040300000102848890B090908888
:101B2000F44F6937100807000000000080403F07AD
:101B3000030303C3331333D316141C0C0B7DC700EC
:101B400000000000000000060F1F1C1C1C1C1C1EB7
:101B50000D00000000070C0E0E0E0E0E0F0E0C00F6
:101B60000000000000000000000080E030D8EC36EB
:101B7000DA7ABABABABAB6B4ACA89830E0000000C3
:101B80000000000080C060BFB18E4C4D508174EDEC
:101B9000C0BE7A7AAA327E620A00BFD0D0B060C0DE
:101BA0007EC3BDB0AF9F1F2F70FBFCFFFFFEFD7B10
:101BB000776F4F6F6F770BB096C86F37180F008035
:101BC00080C060BFC0F8FCFCFC3CCC6CCC2CE9EBCA
:101BD000E3F3F48238EF0000000000000F1930201A
:101BE000232323232321321F01000F181311111166
:101BF00011111011131E0000000000000000000071
:101C000000000000F00CF4F8F0FC04F8F000000014
:101C100000000000000000000000000000000000C4
:101C2000000001867913038B9A0923B22A9CF8805D
:101C3000000000000000000000804020A0601806A6
:101C40000131419E8760180F8B6A9B8463180700DF
:101C5000000000000000008384483F0080403008FE
:101C6000081824C0001EE100000000000000000071
:101C7000000000000F101014161512121C000000B6
:101C80000C0B080A0B0A0A0A09090E0000000000E2
:101C9000000000000000000000F80EF20A060E022C
:101CA000FA060CF800000000000000000000000030
:101CB0000000000000000083CE7986ECFC7465F61D
:101CC000DC4DD563067CC080000000000000C060D1
:101CD000B0D0509CE7F9FECEBE61789FE7F07495D6
:101CE000647B9CE7380F000000000080C74C7BB786
:101CF000C0FF7FBFCF773767DB3FFFE11EF3018176
:101D00008180800000000000001F302F2F2B292A27
:101D10002D2D233E001E1314171514151515161618
:101D2000111F000000000000000000000000000083
:101D30000000000000804020300898909088043C0B
:101D4000D0300000000000000000000000008060B3
:101D5000AE31314941627C930C01599D811AFE01DB
:101D60000000000000000000F0101C0283C2447953
:101D700022A47E40483E35424A360202010000005D
:101D8000000000000000000102020203020404053A
:101D9000070000000000000000000000000000003C
:101DA0000000000000000000000000000000000033
:101DB0000000000000000000000000000000000023
:101DC00000000000000000008080C060B0D8CCF4AB
:101DD000646C6C76FAC22EC8F800000000000000A7
:101DE000000000C0709F51CECEB6BE9D836CF3FE46
:101DF000A6627EE501FE03000000000000F808EE88
:101E0000E3FD7C3DBB86DD5B81BFB7C1CABDB5C903
:101E10007D05060300000000000000010306050523
:101E200005040D0B0B0A080F000000000000000065
:101E300000000000000000000000000000000000A2
:101E40000000000000000000000000000000000092
:101E50000000000000000000000000000000000082
:101E60000000000000000000000000000000000072
:101E70000000000000000080C0202040A02020E0E2
:101E8000C0F008344AF16241677880000000000029
:101E900000007CD29325489324E81116284447C4B7
:101EA000271C201122123EF6FC0700000000000053
:101EB000000103050912355758B0D09887808080FB
:101EC0008080C040300F00000000000000000000D3
:101ED000000000000000000000050F0F0400040FC8
:101EE0000F040000000000000000000000000000DF
:101EF00000000000000000000000000080808080E2
:101F0000808000000000000000000080C06030D031
:101F1000D0B050D0D010380CF6CBB50E9DBE9887FF
:101F20007CC08000000000FE832D6CDAB76CDB17EC
:101F3000EEE9D7BBB83BD8E3DFEEDDEDC10903F82E
:101F40000F000000000003060C1A366DCAA8A74F48
:101F50002F67787F7F7F7F7F3FBFCF701F0100009B
:101F600000000000000000000000000001010F1A46
:101F700010101B0F1B10101B0E00000000000000B3
:101F8000000000F00868481008C88888840204022D
:101F90008488C8F870000000000000000000000005
:101FA000805C6743C08074880B1213147252771ED2
:101FB00013C8799E40A0A0C08000003C424F5065ED
:101FC00035F50F04030203030202020202070DF3B8
:101FD00086CF69371A0A07000000000080403E01E2
:101FE000000000C0301030D8080404020F70C00098
:101FF00000000000000000060911141C141C141E2F
:102000000D00000000070C080A0A0E0A0F0A0C0057
:102010000000000000000000F80CF494B4ECF4346C
:1020200074767BFDFBFD7B7634048CF800000000A9
:102030000000000080C07FA398BC3F7F8B77F4ED49
:10204000ECEB8DAD88E1EC378661BF50503060C05D
:102050007EC3BDB0AF9ACA0AF0FBFCFDFCFCFDFDDF
:10206000FDFDFDF8F20C793096C86535180F00803B
:1020700080C060BFC1FEFFFFFF3FCF6FCF27F7FBE0
:10208000FBFDF08F39E10100000000000F19362E32
:102090002B232B232B21321F01000F18131715158B
:1020A00011151015131E00000000000000000000B4
:1020B0000000000000FEFE82FE82FE82FE000000A4
:1020C0000000000000000000000000000000000010
:1020D00000768E87C6B70E174677FF8E7600000013
:1020E0000000000000000000000000C0304C625101
:1020F000F92221C79F7F7CBFFFA3E09090E0000002
:102100000000000000000000008181414121BD83EA
:1021100041710E0204846919C2320C0000000000F3
:102120000000000000060F1F1E1A1D1D0C000000FD
:1021300000000E0F0E0F0C0E0E0600000000000037
:1021400000000000000000000000FF01017D017D93
:10215000017D01FF00000000000000000000000001
:10216000000000000000FF8971783948F1E8B98863
:10217000007189FF00000000000000000000000066
:10218000E038CEB39DAE06DDDE3860808340005C73
:102190001F686818F0000000000000000080C342C3
:1021A00062A2B2DE427CBE8EF11DCB7B96E63DCDB7
:1021B000731F01000000000000000F1930202125CE
:1021C0002222331F0100001F1110111013111119C9
:1021D0000F0000000000FFFFFFFF3FDFEFF7FBFDF8
:1021E0007D7DBDBDBDDDDDDDDD9DBBB72F5F3F7FEF
:1021F000FFFFFF7FBFDF80BF071BBD0EEF87FBFB2D
:10220000F5C9C9C9FDFD894BCBF3F60CC1FFDFEC65
:10221000EBF7F7F783BC7FFF7EFEFDFCFAFAF6E5ED
:10222000D5D1E5F6FAFAFA00EFDF0F0F0F0F0F0F17
:102230000F0F0F0E0F0E0D0B0B03070707070707F6
:102240000B0D0E0F0F0F17171737377B3B9BC9E985
:10225000B1B1911113B3F7F7AF0F1F3FFFFFFFFFAE
:10226000FFFF828282824222F3FFEF6DABABFFE77A
:10227000EF0D1D1D6C6A9CDDE6B105D2DBFFBEDEF5
:10228000DEEEEFF4F3F7EFEFDFDFBFBFDFBEDCBC66
:10229000DCC7B77BFBFDFEFFFFFF0F0F0F0F0F0F1C
:1022A0000F030F0F0F0F0F0F0F0F0F0F030F0F0F56
:1022B0000C030F0F0F0FFF7FBF7F9FDFEFF3FBFDBF
:1022C000FBFBFBFBF7FBFDFDFDDDBBBBFBCBAB77FE
:1022D000FFFFEF16F9FFCFF7FFFFFB873BDB4D4B0F
:1022E00047CFDF3FFDFF7F2B2DF3FFFE0DF3FB06F6
:1022F000BDA3DFA19E71CFEDF2FF983771707FE330
:10230000CCF0F107E0E9F7FBFCFF0D0C0F0F0F0F0E
:102310000F0F0E0E0D0D0B0B0B0B030B0B0B0B0C02
:102320000F0F0F0F0F0FFFFFFFFFFFFF7FBFDFEF4D
:10233000733377F9FDFBFDFEFD7B37EF9F7FFFFFDA
:10234000FFFFFFFFFFFFFF01FEFFE1DABBA20288F4
:1023500041EFEFE1E8E2E3DAA100FFFFFFFFFFFF5B
:10236000FF7F7F3E310FFFFFFFFCFBF6F5F5F5E544
:10237000070703137BF7E0FFFFFF07090D0E0E0FA2
:102380000F00070B0D0B070B0D0B070808080808BB
:102390000E0E0C09070F7F9FEF6FEFDFBFDFDFDF50
:1023A000EFEFF7FBFDFBFBFDF3EFF7EFCF0FEF1FB9
:1023B000FFFFFC3B97C6D4FEFFFFAFEFBCA199899E
:1023C000C13FBFDF9F010959C07F68F7EF1FFFF0D2
:1023D000E7CB1F2F5F736DDEBE7E7DFDFCFBE3EB65
:1023E000EBE37D7C3D1ECFE0F7F80F0703080E0FEF
:1023F0000F0F0E0E0E0E0E0E0E0E0E0E0E0E0F0FF9
:102400000E0803070F0FFFFFFFFFFC03A756205026
:10241000205020502757275721502050A000FCFF64
:10242000FFFFFFFFFF4793D86C26C2F252424232B1
:10243000F2424252F2C2266CD89047FFFFFFFFFFE4
:10244000FFFC7BBBD89953EF1F7E2FA8AB2B7E1FC1
:10245000EF5399D8BB7BFCFFFFFF0F0F030C0F0F4F
:102460000F0F080B090C0C0307030C090B080F0FC7
:102470000F0F0C030F0F0000000000E0F0F0F8FC5D
:10248000FC00000000000000000000000000000050
:1024900000010303070F0F00000000000000000010
:1024A000000000000000F018080C060202FE000008
:1024B0000000000000000000000000000306040C03
:1024C0001810101F000000000000000000000000B5
:1024D000000000E0F0F0F8FCFC00E008F204F80076
:1024E000000000000000000000010303070F0F00C0
:1024F0000104130807000000000000000000F018AD
:10250000080C060202FE1CF70DFB06FC0000000092
:10251000000000000306040C1810101F0E3B2C379F
:10252000180F0000000000003CA6A2F25272068CB8
:10253000F8FE020202626202060CF80000001F119F
:102540001010121213131E1F1010101C0404060387
:1025500001000000784CC60202FE0000FE020202EA
:10256000626202060CF8000000001E121310101325
:10257000121E1F1010101C040406030100000000AE
:1025800000181C0C8C8CF8700000FCFCFC9C9CFC63
:10259000F8F000000000000E0F0F0D0D0C0C0000F5
:1025A0000F0F0F030303010000000000003038FC90
:1025B000FC00000000FCFCFC9C9CFCF8F00000000F
:1025C0000000000C0C0F0F0C0C00000F0F0F03038A
:1025D000030100000000FEFFFFFFFFFFFFFFFFFF02
:1025E000FFFFFFFFFFFFFFFFFFFFFFFFFFFFFFFEFC
:1025F0007FFFFFFFFFFFFFFFFFFFFFFFFFFFFFFF6B
:10260000FFFFFFFFFFFFFFFFFF7F000000000080D4
:102610008080C0C0C0C0C0C080000080808080803A
:102620000000000080C0C0C0C0C0C0C0C0C0E0F09A
:10263000F81C0C0C0C1CF8F0F8FCCE868686CEFC40
:10264000F8E0C08080008080808080000000000072
:1026500000000000000000000000FCFEFFC30301BA
:1026600001010030303030FD1F0703030321310129
:102670008183838F7F21202040C8CC0C10113FF82C
:10268000F80000000000F8F8FF0300000000FFF170
:10269000C00000010F1F0703038343370F0E0E0610
:1026A000868E0C0C1838F0C0800000073FFFFFF04A
:1026B000C0808080C4FCFCFF7FFCF8F0F0F0F1F1FA
:1026C00030989C9F9F9C1C1C9C9C1C1C1C1C9E9FAF
:1026D0009F9E1C1C1C9E1F1F1F9C1C1C9C9E9F9F22
:1026E0009F9F3830F0F8FCFE7FFFFCF0E0C0C0C0D8
:1026F000C4C8C8E8F8F8FF7F3F00000000010307E6
:102700000F0F0F0F0F0703000000000101FFFF80F4
:10271000007FFFFF1B0B01007FFFFF003E7FF3E305
:10272000F377F70000FFFF1C1CFFFF000303FFFF10
:1027300003030000FFFFFF000000010303070F0F6A
:102740000F0F070703010000000000000000000059
:10275000000000000000000000000000000F1F3F0C
:102760003F7E7C7C7C7C7C7C7C7C7C7C7C7C7C7CE4
:102770007C7C7C7C7C7C7C7C7C7C7C7C7C7C7C7C99
:102780007C7C3E3F1F0F03000000000000000000A3
:102790000000000000000000000063726169742EF8
:1027A0006E65740040637261697400486F6C6D659A
:1027B00073004A6F6E617468616E00458A15AA15D0
:1027C000AAD56A342821321D0A0C06030207022307
:1027D00041A0418040814020804080402008C77D4A
:1027E000A255A251A8158844A251AA54A851820505
:1027F000FF00004180800080E0F0F0F0F0E06060D9
:102800006068EDE4E3E0E06172E102E1321AAF11E9
:1028100088548A452A059245A241A055AA55AA5531
:10282000BFE0000000003CFEFFFFFF1DEC3637F765
:10283000F7EE1FFF3FDF2E37F6EE1C037E55CAC5AD
:10284000A251A854AA552A158A452251A254A0552E
:10285000FEC3BC66400038DF7FBFFFFFFE7D7D7D8D
:10286000FDFE3F7FFFF06D1DBDFEFFE0833FC07F9B
:10287000A255A2512804A251A854AA11A215A2C57A
:102880006A4563416B5E7871A64B8D979C38312306
:1028900006464D4D6D727F6F1F370F1DCBE07F5584
:1028A0006A4540C08AC56AB5DAEDCA3DCEF3FDFE81
:1028B000F8877FFFFFFFFFC0BFBEBDDB57A7CFB7C5
:1028C0008BFAF676A6CA76EA9C5FDFC0FEFEFFFFB3
:1028D000FFFF0FB6B9FBF8F3F7FFF8010204081089
:1028E00020408000000000003E5B4F5B3E3E6B4F8F
:1028F0006B3E1C3E7C3E1C183C7E3C181C577D5792
:102900001C1C5E7F5E1C00183C1800FFE7C3E7FF3D
:102910000018241800FFE7DBE7FF30483A060E26D0
:1029200029792926407F050507407F05253F5A3C28
:10293000E73C5A7F3E1C1C08081C1C3E7F14227F6B
:1029400022145F5F005F5F06097F017F0066899543
:102950006A606060606094A2FFA29408047E04082C
:1029600010207E201008082A1C08081C2A08081EAF
:10297000101010100C1E0C1E0C30383E3830060E95
:102980003E0E06000000000000005F00000007008F
:102990000700147F147F14242A7F2A12231308644B
:1029A0006236495620500008070300001C224100EF
:1029B0000041221C002A1C7F1C2A08083E0808002F
:1029C00080703000080808080800006060002010CF
:1029D0000804023E5149453E00427F400072494989
:1029E00049462141494D331814127F10274545456A
:1029F000393C4A494931412111090736494949368B
:102A0000464949291E00001400000040340000001F
:102A10000814224114141414140041221408020151
:102A20005909063E415D594E7C1211127C7F49497D
:102A300049363E414141227F4141413E7F4949491A
:102A4000417F090909013E414151737F0808087F10
:102A500000417F41002040413F017F081422417F17
:102A6000404040407F021C027F7F0408107F3E41AF
:102A700041413E7F090909063E4151215E7F091906
:102A80002946264949493203017F01033F4040401E
:102A90003F1F2040201F3F4038403F63140814630D
:102AA00003047804036159494D43007F41414102C9
:102AB00004081020004141417F040201020440400B
:102AC000404040000307080020545478407F2844C9
:102AD00044383844444428384444287F38545454B3
:102AE0001800087E090218A4A49C787F08040478C2
:102AF00000447D40002040403D007F1028440000FD
:102B0000417F40007C047804787C080404783844D1
:102B1000444438FC1824241818242418FC7C080485
:102B20000408485454542404043F44243C404020A6
:102B30007C1C2040201C3C4030403C442810284451
:102B40004C9090907C4464544C4400083641000002
:102B500000770000004136080002010204023C2612
:102B600023263C1EA1A161123A4040207A385454D9
:102B7000555921555579412154547841215554785E
:102B80004020545579400C1E5272123955555559F2
:102B9000395454545939555454580000457C410017
:102BA00002457D420001457C40F0292429F0F028AF
:102BB0002528F07C545545002054547C547C0A0947
:102BC0007F4932494949323248484832324A4848B6
:102BD000303A4141217A3A42402078009DA0A07DC0
:102BE00039444444393D4040403D3C24FF2424487E
:102BF0007E4943662B2FFC2F2BFF0929F620C08826
:102C00007E090320545479410000447D41304848F6
:102C10004A32384040227A007A0A0A727D0D193110
:102C20007D2629292F28262929292630484D40206C
:102C3000380808080808080808382F10C8ACBA2F48
:102C4000102834FA00007B000008142A14222214F1
:102C50002A14089500220095AA005500AAAA55AA90
:102C600055AA000000FF00101010FF00141414FFFC
:102C7000001010FF00FF1010F010F0141414FC00EE
:102C80001414F700FF0000FF00FF1414F404FC14F8
:102C90001417101F10101F101F1414141F001010F1
:102CA00010F0000000001F101010101F1010101066
:102CB000F010000000FF101010101010101010FF86
:102CC00010000000FF140000FF00FF00001F10179D
:102CD0000000FC04F414141710171414F404F40086
:102CE00000FF00F714141414141414F700F714144C
:102CF00014171410101F101F141414F4141010F0D3
:102D000010F000001F101F0000001F14000000FC46
:102D1000140000F010F01010FF10FF141414FF1432
:102D20001010101F00000000F010FFFFFFFFFFF069
:102D3000F0F0F0F0FFFFFF0000000000FFFF0F0FBA
:102D40000F0F0F38444438447C2A2A3E147E020276
:102D50000606027E027E0263554941633844443CC4
:102D600004407E201E2006027E020299A5E7A59956
:102D70001C2A492A1C4C7201724C304A4D4D30308D
:102D800048784830BC625A463D3E494949007E0178
:102D900001017E2A2A2A2A2A44445F444440514A97
:102DA000444040444A51400000FF0103E080FF00DE
:102DB0000008086B6B083612362436060F090F061A
:102DC000000018180000001010003040FF01010042
:102DD0001F01011E00191D1712003C3C3C3C000065
:102DE00000000000000000240027002A002D003011
:102DF0000000000000250028002B002E00310004F8
:102E000008020110408040102040804080080204E9
:102E10000180402010020110801020404020040456
:102E20000404040304050202020204030202020273
:102E3000060606060606040402020204040601153C
:102E400001260137014A015D01720188019F01B825
:102E500001D201EE010B022A024B026E029302BA6A
:102E600002E40210033F037003A403DC03170455BC
:102E7000049704DD0427057505C80520067D06E0D6
:102E8000064907B8072D08A9082D09B9094D0AEA0E
:102E90000A900B400CFA0CC00D910E6F0F5A105394
:102EA000115B1272139A14D41520178018F519802B
:102EB0001B231DDE1EB420A622B524E4263429A738
:102EC0002B402E0031EA330037453ABC3D68414C77
:102ED000456B49C84D68524F57805C006210111213
:102EE00013151617181A1C1D1F21232527292C2EF0
:102EF0003134373A3E4145494E52575C62686E75EF
:102F00007B838B939CA5AFB9C4D0DCE9F7080B0099
:102F1000020202010009040000010202000005246F
:102F20000010010524010101042402060524060005
:102F3000010705810310004009040100020A000096
:102F4000000705020240000007058302400000045C
:102F500003090412010002EF020140412336800000
:102F6000010102030141726475696E6F204C4C438C
:102F70000041726475696E6F204C656F6E6172649A
:102F80006F00182F11241FBECFEFDAE0DEBFCDBFD8
:102F900011E0A0E0B1E0E2ECF1E602C005900D9294
:102FA000A435B107D9F726E0A4E5B1E001C01D9230
:102FB000A732B207E1F717E1C2ECD7E104C02197CD
:102FC000FE010E94D430C13CD107C9F70E945124B0
:102FD0000C94DF300C9400004091910150919201CB
:102FE00020918F013091900142175307B4F49091D2
:102FF000E8009570E1F39091E80092FD19C080938C
:10300000F100809191019091920101968F7399271F
:10301000892B19F48EEF8093E800809191019091B3
:1030200092010196909392018093910181E008951D
:1030300080E00895DF92EF92FF920F931F93CF935A
:10304000DF93D82E8A017B01E40EF51EEB01CE152D
:10305000DF0571F0D7FE03C0FE01849101C08881B5
:103060000E94EC1721968111F2CF8FEF9FEF01C0E4
:10307000C801DF91CF911F910F91FF90EF90DF90EA
:103080000895615030F02091F100FC0120830196F9
:10309000F8CF289884E6809394010895CF92DF9228
:1030A000EF92FF920F931F93CF93DF936C017A01FE
:1030B0008B01C0E0D0E0CE15DF0589F0D8016D911D
:1030C0008D01D601ED91FC910190F081E02DC601BA
:1030D0000995892B11F47E0102C02196ECCFC7011E
:1030E000DF91CF911F910F91FF90EF90DF90CF90E4
:1030F0000895CF93DF931F92CDB7DEB76983DC01CC
:10310000ED91FC910280F381E02D41E050E0BE01A1
:103110006F5F7F4F09950F90DF91CF91089583E006
:103120008093E9008091F200882319F08AE380936C
:10313000E8000895FC018485958597FD0BC09FB735
:10314000F89482E08093E9008091F2009FBF90E0C4
:10315000019608959FB7F89482E08093E9008091EA
:10316000F2009FBF90E00895CF92DF92EF92FF921E
:103170001F93CF93DF93E82FF0E0E15EFE4F1081C5
:10318000E62FF0E0603330F4E352F14DE491CE2FBE
:10319000D0E006C0EE0FFF1FE352F24DC591D4916F
:1031A0006E01E12CF12C60E074E284EF90E0A70165
:1031B00096010E947130DA01C9010197A109B10994
:1031C000009721E0A207B10578F060E970ED83E097
:1031D00090E0A70196010E947130DA01C9010197C0
:1031E000A109B10923E001C021E01130C9F0133079
:1031F00051F530919100387F232B209391009093CB
:10320000990080939800D0938801C093870181E052
:10321000809386018091710082608093710013C059
:103220003091890131110FC030918100387F232BFB
:1032300020938100909389008093880080916F0093
:10324000826080936F00DF91CF911F91FF90EF908C
:10325000DF90CF900895E82FF0E0E15EFE4F80818F
:10326000813019F0833089F00895809189018111AE
:1032700022C080916F008D7F80936F0090917301C9
:10328000E0917101F09172010CC010928601809161
:103290008501811110C090918301E0918101F0912D
:1032A00082018081282F30E0892F90E080959095D1
:1032B000822393238083089580915B01089508956C
:1032C000089580E090E008950E94DA300F931F93F4
:1032D000CF93DF931F92CDB7DEB782E0898342E4BC
:1032E00050E06DE07FE280E80E941A180E943D24C1
:1032F000DC0112960D911C9113970115110569F0CF
:10330000D801ED91FC910280F381E02DBE016F5F49
:103310007F4FC801099597FF07C089810F90DF9102
:10332000CF911F910F910895F80100851185E5CF88
:103330000E94022490E00895CF93DF931F92CDB7AF
:10334000DEB7FC018485958597FD05C02FEF3FEF23
:10335000358724870BC0CE0101960E941324019764
:1033600019F4898190E002C08FEF9FEF0F90DF91F9
:10337000CF9108950F931F93CF93DF931F92CDB7F3
:10338000DEB78C01FC018485958597FF0EC0CE01C8
:1033900001960E941324019719F4298130E002C09C
:1033A0002FEF3FEFF80135872487F8018485958555
:1033B0000F90DF91CF911F910F9108951F920F925F
:1033C0000FB60F9211248F939F938091E1009091FB
:1033D000E100937F9093E10083FF0FC01092E9001A
:1033E00091E09093EB001092EC0092E39093ED004B
:1033F0001092950198E09093F00082FF20C093E036
:103400009093E9009091F200992319F09AE3909338
:10341000E80090919301992339F090919301915094
:1034200090939301992389F190919401992339F014
:1034300090919401915090939401992341F184FFCC
:1034400010C08091E2008E7E81608093E2008091C6
:10345000E1008F7E8093E100809155018E7E806136
:1034600011C080FF16C08091E2008E7E8061809343
:10347000E2008091E1008E7E8093E1008091550111
:103480008E7E81608093550104C05D9ACDCF289ACD
:10349000D6CF9F918F910F900FBE0F901F901895D0
:1034A0001F920F920FB60F921124CF92DF92EF92DC
:1034B000FF920F931F932F933F934F935F936F93BD
:1034C0007F938F939F93AF93BF93EF93FF93CF938C
:1034D000DF93CDB7DEB76C97DEBFCDBF1092E900AA
:1034E0008091E80083FFEDC168E0CE0145960E941F
:1034F000411882EF8093E8008D8987FF05C0909185
:10350000E80090FFFCCF03C09EEF9093E800982F57
:10351000907609F0C6C09E892F89188D91110CC034
:10352000803829F4809156018093F10002C01092F6
:10353000F1001092F10048C1422F50E0512B913020
:1035400051F4811141C14130510509F03DC18091D3
:1035500056018D7F0BC0933061F4811135C141302C
:10356000510509F031C18091560182608093560166
:103570002BC1953041F48091E80080FFFCCF20689A
:103580002093E30021C1963009F05FC0EB8CFC8CE6
:103590001092E9001092920110929101123091F56F
:1035A0001092900110928F010E94661999E0BE015D
:1035B0006F5F7F4FDB01E92F1D92EA95E9F7998351
:1035C0001A8391E09E8390EA98879AEF99872091D9
:1035D000910130919201275F3F4F3C832B838D8374
:1035E0001092E9001092920110929101F0929001D4
:1035F000E0928F0149E050E080E00E941A180E949A
:103600006619E2C0F0929001E0928F010E943D2481
:10361000DC011296ED90FC901397E114F10409F48B
:10362000C0C0D701ED91FC910480F581E02DBE0171
:103630006B5E7F4FC7010995009719F00CF0C4C06D
:10364000C7C0F701E084F184E8CF973009F4C0C027
:10365000983021F481E08093F100B6C0993009F0F0
:10366000B3C0837009F0B4C0E2E2F1E081E021E090
:1036700036E39081992361F08093E9002093EB0079
:1036800091919093EC003093ED008F5F873089F734
:103690008EE78093EA001092EA008F89809395016B
:1036A00093C08B8D9C8D1092E90010929201109224
:1036B00091019093900180938F01898D811156C063
:1036C0008E899D89913A59F4813209F081C047E091
:1036D00050E067E071E080E00E941A1875C09132F6
:1036E00009F076C0833289F4888D90E0982F88277E
:1036F0002F89822BA0E0B0E0809303019093040116
:10370000A0930501B09306015FC0803269F48091F7
:10371000E80082FFFCCF67E087E091E00E9441185B
:103720008BEF8093E80006C0823209F04DC08F898C
:1037300080930E0180915401882319F0EEEFFAE096
:1037400002C0E0E0F8E08091070190910801A091AB
:103750000901B0910A01803B9440A105B10509F02F
:103760007BC080910E0180FF93C076C00E943D24F3
:10377000DC0112960D911C9113970115110541F171
:10378000D801ED91FC910190F081E02DBE016B5EBE
:103790007F4FC8010995811117C0F8010085118577
:1037A000ECCF113009F44EC0133091F48F89882387
:1037B00009F445C0823081F440E860E181E79FE28E
:1037C0000E94972E882321F08EEF8093E80079C025
:1037D00081E28093EB0075C0813029F440E86BE012
:1037E00085E69FE2EDCF833099F70E943D24DC010E
:1037F0001296ED90FC9013978E010F5F1F4F68019A
:10380000E114F10479F0D701ED91FC910680F78184
:10381000E02DB801C7010995080F111DF701E084DB
:10382000F184EECFD8011C92F60101900020E9F757
:103830003197BF016C197D0940E0C601C1CF6FE42B
:103840007FE202C063E57FE26115710509F2FB01C9
:10385000449150E080E840CF0FB6F894A89580914D
:103860006000886180936000109260000FBEA89590
:10387000EE3F2AE0F20739F08091FE0A9091FF0AAC
:1038800091838083A1CF1092FF0A1092FE0A9CCFF1
:10389000EE3F8AE0F80731F0808191819093FF0A32
:1038A0008093FE0A87E797E7918380839BE088E116
:1038B0000FB6F894A895809360000FBE90936000B7
:1038C00083CF6C960FB6F894DEBF0FBECDBFDF91ED
:1038D000CF91FF91EF91BF91AF919F918F917F9188
:1038E0006F915F914F913F912F911F910F91FF9099
:1038F000EF90DF90CF900F900FBE0F901F90189514
:103900003FB7F89480918B0190918C01A0918D012B
:10391000B0918E0126B5A89B05C02F3F19F00196E6
:10392000A11DB11D3FBFBA2FA92F982F8827820F45
:10393000911DA11DB11DBC01CD0142E0660F771F95
:10394000881F991F4A95D1F708958F929F92AF9241
:10395000BF92CF92DF92EF92FF926B017C010E94A7
:10396000801C4B015C01C114D104E104F104F1F0AD
:103970000E94801CDC01CB0188199909AA09BB09A6
:10398000883E9340A105B10570F321E0C21AD10829
:10399000E108F10888EE880E83E0981EA11CB11C96
:1039A000C114D104E104F10419F7DDCFFF90EF90C9
:1039B000DF90CF90BF90AF909F908F9008958F929F
:1039C0009F92AF92BF92CF92DF92EF92FF920F93AE
:1039D0001F93CF93DF935C016B017A0180910E01FD
:1039E000882309F45BC080919501882309F456C0AF
:1039F0008091550180FF05C08091E0008260809336
:103A0000E000E70110E00AEF83E0882E9AE3992EA8
:103A10002097D9F10E94022481110AC0015009F4B3
:103A20003DC061E070E080E090E00E94A51CF0CF16
:103A3000282F30E0C217D3070CF48C2F4FB7F8941F
:103A40008092E9009091E80095FF1DC0282F30E09A
:103A5000C21BD30BF601982F915020F081918093D7
:103A6000F100FACFC20ED31E112319F09092E80094
:103A700009C08091E80085FD06C09092E80011E041
:103A8000209709F010E04FBFC3CF1111C3CF5D984D
:103A900084E6809393011E141F0444F081E090E0BB
:103AA000F5019383828380E090E001C0C701DF913C
:103AB000CF911F910F91FF90EF90DF90CF90BF902B
:103AC000AF909F908F9008951F920F920FB60F9214
:103AD00011242F933F938F939F93AF93BF93809124
:103AE000570190915801A0915901B0915A0130911C
:103AF0008A0123E0230F2D3720F40196A11DB11D6B
:103B000005C026E8230F0296A11DB11D20938A014E
:103B10008093570190935801A0935901B0935A0193
:103B200080918B0190918C01A0918D01B0918E01BB
:103B30000196A11DB11D80938B0190938C01A093E0
:103B40008D01B0938E01BF91AF919F918F913F9165
:103B50002F910F900FBE0F901F9018951F920F92EC
:103B60000FB60F9211242F933F934F935F936F9350
:103B70007F938F939F93AF93BF93CF93DF93EF93F5
:103B8000FF9380918601882349F0809185018111FE
:103B900005C080918401882309F4ABC08091800125
:103BA000882309F4B6C080917C0190917D01A09199
:103BB0007E01B0917F01892B8A2B8B2B09F4A9C040
:103BC00080917C0190917D01A0917E01B0917F0157
:103BD0000197A109B10980937C0190937D01A09385
:103BE0007E01B0937F01892B8A2B8B2B09F091C02A
:103BF000D1E0E0917A01F0917B019F012F5F3F4F6F
:103C000030937B0120937A018491982F907FC82F65
:103C1000CF70903821F48C2F0E942B19EACF903965
:103C2000F9F4E091E605F091E70509958D27809379
:103C30008401E0917A01F0917B01CF01019690938C
:103C40007B0180937A01649180917901C81788F68D
:103C5000C13009F058C0809178018111CACF53C09A
:103C600097FD3AC03296F0937B01E0937A01F90117
:103C7000249130E0382BA0918701B09188010E94F7
:103C8000C5306C507E4F8F4F9F4F28EE33E040E0A1
:103C900050E00E94A33020937C0130937D0140933B
:103CA0007E0150937F0180917C0190917D01A091D4
:103CB0007E01B0917F01892B8A2B8B2B51F581E0FE
:103CC00090E0A0E0B0E080937C0190937D01A09310
:103CD0007E01B0937F011DC0903E29F410927B01BC
:103CE00010927A0186CF903F09F083CF1092800125
:103CF00010C080918301E0918101F0918201908157
:103D0000892780834BCF67FD74CF8C2F0E94B41816
:103D100070CFFF91EF91DF91CF91BF91AF919F91C4
:103D20008F917F916F915F914F913F912F910F9064
:103D30000FBE0F901F9018951F920F920FB60F9203
:103D400011242F933F938F939F93AF93BF93EF9340
:103D5000FF9380918901882309F44FC080917401F9
:103D600090917501A0917601B0917701892B8A2BF2
:103D70008B2B51F180917301E0917101F0917201EF
:103D80009081892780838091740190917501A09121
:103D90007601B0917701181619061A061B06D4F59C
:103DA0008091740190917501A0917601B091770195
:103DB0000197A109B1098093740190937501A093B3
:103DC0007601B093770126C0109285011092890187
:103DD00080916F008D7F80936F0090917301E091CF
:103DE0007101F09172018081282F30E0892F90E0DD
:103DF00080959095822393230CC08091840181113A
:103E000009C080917301E0917101F091720190817C
:103E100089278083FF91EF91BF91AF919F918F91FF
:103E20003F912F910F900FBE0F901F90189590917A
:103E30007901923009F471C0292F30E0F901E15E77
:103E4000FE4F4081F901E159FE4F8083913031F4FA
:103E500020916F01281302C0909378019F5F909387
:103E6000790190E0FC01E25EF14D2491FC01E1500A
:103E7000F24D849130E0220F331FF901EF50F24DE3
:103E800065917491F901ED51F24DA591B4919C9118
:103E9000982B9C93413019F04330D9F008959091BC
:103EA0006400977F909364001092800010928100CC
:103EB0009091810098609093810090918100916031
:103EC00090938100709372016093710180937301EC
:103ED000089590916500977F9093650010929000EF
:103EE0001092910090919100986090939100909120
:103EF0009100916090939100709382016093810191
:103F00008093830180917901882321F06CE380E024
:103F10000E94B41880E00C942B1908952D9A0895EE
:103F2000BC0180E090E00C94A51C8FB12CB193B142
:103F300030E02095309520743327A90123E0559572
:103F400047952A95E1F7292F30E02095309520718B
:103F500033273595279535952795242B8095807F98
:103F6000822B089583B7817F83BF83B7816083BF2E
:103F7000889583B78E7F83BF08958EBD00000DB4F2
:103F800007FEFDCF089510925B013E983F9808957B
:103F90003E9A3F9A81E080935B010895FC01840F73
:103FA000911D18161906E4F5E038F105CCF5F7FF78
:103FB00002C0E0E0F0E08138910514F080E890E084
:103FC000382F3E1BAB0177FF02C0495F5F4F83E094
:103FD000559547958A95E1F75695542F442757955F
:103FE0004795E40FF51FEA56FE4F6770772781E08B
:103FF00090E001C0880F6A95EAF7482F222349F024
:10400000213071F4315020F08081842B8193FACFDC
:1040100008958095315020F0908198239193FACFA4
:10402000089560387105D0F440345105B8F4EBEDD3
:10403000F8E280E1849FD001A0781124A60F477098
:10404000E40FF11D8491AA56BE4F222319F06C9102
:10405000862B03C080956C9186238C9308952F92B4
:104060003F924F925F926F927F928F929F92AF9208
:10407000BF92CF92DF92EF92FF920F931F93CF9355
:10408000DF93CDB7DEB729970FB6F894DEBF0FBE2A
:10409000CDBFFC016A3069F4248D808D918D38E0AC
:1040A000239F800D911D1124918F808F178A168A6E
:1040B000AAC06D3009F4A7C099878887F48C338C27
:1040C000228C608C718C0689178900381105C4F028
:1040D000A885B9855C962C915C97422F50E0569646
:1040E0008D919C915797B6E02B9F800D911D1124C7
:1040F000E885F985978B868B258D21116EC083C04D
:10410000F0E46F16710424F7C80125E0F29E800DDB
:10411000911D112418161906DCF68F2D90E09C8352
:104120008B83C301A8E0FA9E800D911D11241816FF
:10413000190674F6B5E06B9FB0011124FB01ED5137
:10414000F74DFA83E98330E08885998504969E834C
:104150008D83E981FA81E490353009F4E12C430143
:1041600088E0482EE0FC02C0532C01C0522C5110B4
:104170000BC0321009C0E6944A948B819C81880E52
:10418000991E4110EFCF1BC068018C2D801B8F152D
:1041900090F754018A2D88198F1568F4252DA501F3
:1041A000B6018D819E813F830E9411209FEFA91A45
:1041B000B90A3F81EFCFAFEFCA1ADA0AE6CF3F5F05
:1041C000EB81FC810E0F1F1F89819A8101969A83D2
:1041D0008983363009F0BDCF7BCF6AEF640390014D
:1041E000659F300D112420583F4F281739075CF484
:1041F000A885B985ED91FC9111970190F081E02D92
:104200006AE0CD01099581E090E029960FB6F89417
:10421000DEBF0FBECDBFDF91CF911F910F91FF90F9
:10422000EF90DF90CF90BF90AF909F908F907F9056
:104230006F905F904F903F902F9008954F925F92B4
:104240006F927F928F929F92AF92BF92CF92DF92A6
:10425000EF92FF92CF93DF9320915B01222309F429
:104260006FC04A015B01EC01E091E605F091E705C2
:104270000995882309F464C080917901823008F49B
:104280005FC081E08093890180916E0180938501F8
:104290002E01612C712C60E072E18AE790E0A301AD
:1042A00092010E94713069017A0181E0C81AD10837
:1042B000E108F108C114D10481E0E806F104F0F14D
:1042C00068E478EE81E090E0A30192010E947130F1
:1042D00069017A0181E0C81AD108E108F10893E088
:1042E00080918100887F892B8093810081149104C3
:1042F000A104B10471F0DE01AA0FBB1FA501940156
:104300000E94903028EE33E040E050E00E94A3305D
:1043100003C02FEF3FEFA901D0928900C09288001F
:104320002093740130937501409376015093770187
:1043300080916F00826080936F0002C091E0D0CFC7
:10434000DF91CF91FF90EF90DF90CF90BF90AF9033
:104350009F908F907F906F905F904F900895CF9334
:10436000C82F88E00E944823882351F044E650E09B
:1043700060E070E080E991E00E941E21C0935C0142
:10438000CF9108952F923F924F925F926F927F92BA
:104390008F929F92AF92BF92CF92DF92EF92FF9255
:1043A0000F931F93CF93DF93CDB7DEB760970FB610
:1043B000F894DEBF0FBECDBFED82CA86C22ED12CCF
:1043C000FC01EC0DFD1DF7FD4AC1803891050CF094
:1043D00046C1FB01E00FF11DF7FD41C160347105DD
:1043E0000CF03DC1DB0177FF04C0AA27BB27A61B49
:1043F000B70BA770BB27FB0177FD379613E0F59548
:10440000E7951A95E1F777FF07C0319768E070E00C
:104410004B018A1A9B0AD401A02EA694A694A694B6
:10442000B12C077019F00FEFA01AB00ABF01F69572
:10443000FE2FEE27F795E795E80FF91F8F010A5633
:104440001E4F1E870D874501860E971E998688860A
:10445000612C712C30E08901015011091C870B87F8
:1044600028E030E049018A1A9B0A9F828E822885C3
:1044700039856217730709F4F2C06830710509F4D1
:10448000EEC06F3F0FEF70070CF4DAC00D851E858C
:1044900000581F4F4D845E8412015C824B821A8348
:1044A00009837801A12CB12CAC14BD040CF0C8C058
:1044B0002A85222329F02B853C852A193B0901C036
:1044C0009501F901E80FF91FE038F1050CF0B8C0CB
:1044D000F7FD9BC06F3FEFEF7E0709F4BCC04901B9
:1044E000860C971CFD81F130B1F4F401E40FF51F47
:1044F000E491F0E04F010A2E02C0880C991C0A9446
:10450000E2F7988A8F86F1019080EF85F889E92992
:104510004F01F10133C0FD81F11119C0F401E40F25
:10452000F51FE491F0E00A2E02C0EE0FFF1F0A947F
:10453000E2F74F0180949094988A8F86F2018080F0
:10454000912CEF85F8898E229F22F20117C0F40189
:10455000E40FF51FE491F0E04F010A2E02C0880C31
:10456000991C0A94E2F7988A8F86EB81FC819080EF
:10457000EF85F889E9254F01EB81FC818082109756
:1045800009F443C06730710509F43FC04901860C46
:10459000971C2D81213089F4F401E40FF51FE4917B
:1045A0002E2F30E049010E8002C0959487940A9422
:1045B000E2F7F8012081822A27C02D81F401E40F5F
:1045C000F51F211113C0E4912E2F30E00E8002C0A0
:1045D000359527950A94E2F7490180949094F70164
:1045E000208130E02821392120830FC0E4912E2F33
:1045F00030E049010E8002C0959487940A94E2F756
:10460000E981FA81208182268082FFEFAF1ABF0AFA
:104610000F5F1F4F2FEFE21AF20A29813A812F5FB5
:104620003F4F3A8329832B813C812F5F3F4F3C834F
:104630002B833FEF231A330AEFEF4E1A5E0A34CF73
:104640006F5F7F4F0D851E8500581F4F1E870D879A
:104650006C0C7D1C0CCF109709F098CFD6CF6096CC
:104660000FB6F894DEBF0FBECDBFDF91CF911F9183
:104670000F91FF90EF90DF90CF90BF90AF909F9001
:104680008F907F906F905F904F903F902F90089504
:1046900020910706282329F490910606982381E0AB
:1046A00009F480E0089580E0E6E9F1E081118FEF00
:1046B000002481938193819381930394D1F708958A
:1046C000809196018EBDE7E9F1E081910DB407FE7E
:1046D000FDCF8EBD85E0E639F807B9F70DB407FECA
:1046E000FDCF08950F931F93CF93DF938C01C0E00C
:1046F000D0E0F801EC0FFD1F6491662371F0E091AA
:10470000FD05F091FE050190F081E02D8DEF95E023
:104710000995892B11F02196ECCFCE01DF91CF9135
:104720001F910F9108958F929F92AF92BF92CF9257
:10473000DF92EF92FF920F931F93CF93DF937C0151
:10474000EB01142FD22E6034710518F4202F0E9433
:10475000CE1F4E018D0C911CB40161507109603463
:10476000710528F4202F412FC7010E94CE1FD7FFCB
:1047700002C0C0E0D0E06E01540181E488169104CB
:104780001CF080E4A82EB12CCA14DB045CF4202FAA
:10479000A601B70181E096E00E9411208FEFC81AB0
:1047A000D80AEACFE10EF11C81E0E81AF108CA1537
:1047B000DB054CF4202FAE01B70181E096E00E94AA
:1047C00011202196F4CFDF91CF911F910F91FF908F
:1047D000EF90DF90CF90BF90AF909F908F90089513
:1047E000009769F0FC0101900020E9F73197AF01D3
:1047F000481B590BBC018DEF95E00C944E1880E0DE
:1048000090E008952FB7F89483E08093E9009091A9
:10481000E800892F807295FF04C09091F20080E437
:10482000891B2FBF0895FC0180919501811103C060
:104830008FEF9FEF08959FB7F89482E08093E9008F
:104840002091F20030E01216130614F421E030E05B
:104850002115310559F0289884E6809394018091C0
:10486000F10080838091F200882319F09FBFC90175
:1048700008958BE68093E800F9CF80911F0681119F
:104880000DC082E080931B0684E080931C0610928A
:104890001E0610921D0681E080931F068BE196E0B4
:1048A0000895CF93DF9300D01F92CDB7DEB77894F1
:1048B00084B5826084BD84B5816084BD85B5826025
:1048C00085BD85B5816085BD80916E0081608093D6
:1048D0006E0010928100809181008260809381003F
:1048E000809181008160809381008091800081604F
:1048F00080938000809191008260809391008091EC
:1049000091008160809391008091900081608093FC
:1049100090008091C10084608093C1008091C100AB
:1049200082608093C1008091C10081608093C1004A
:104930008091C30081608093C3008091C000826039
:104940008093C0008091C20081608093C2008091FA
:104950007A00846080937A0080917A0082608093EC
:104960007A0080917A00816080937A0080917A0049
:10497000806880937A0010929501109256011092EF
:1049800055018091D70081608093D70080EA8093A1
:10499000D80089B5806189BD89B5826089BD09B4B7
:1049A00000FEFDCF61E070E080E090E00E94A51C79
:1049B0008091D8008F7C80618093D8008091E00046
:1049C000807F8093E0008091E1008E7E8093E10003
:1049D0008DE08093E200559A209AEEEFFFE78591F3
:1049E00094918B3F9C4D19F481E08093540181ECAC
:1049F00080937C0085B1806F85B9249884B1866EE0
:104A000084B95E9A5F988AB1806D8AB9769A6E98F9
:104A100081B3806F81BB899880B38D7080BB80E546
:104A20008CBD81E08DBD85E090E00E94901F5F9A73
:104A300085E090E00E94901F5E985C98FCE5EF2E68
:104A4000F1E0FF2E1DE01E0DF70184910E94BD1FB5
:104A5000FFEFEF1AFF0A1E11F7CF5C9A81E88093EF
:104A6000640081E08093650000E014E080E00E9433
:104A7000BD1F01501109D1F70E94951F87FF1FC06C
:104A80005C9885EA0E94BD1F5C9A2E982F982D98FD
:104A9000809164008062809364000E94B21FFDCF09
:104AA0002D980E94951F8478843871F00E94951F7C
:104AB0008471843131F188EC90E00E94901F0E9453
:104AC000951F82FDEDCF3AC00E948E1F88EC90E0CA
:104AD0000E94901F2F9882E090E00E945B308F3FF1
:104AE00029F06FEF82E090E00E94633084EF91E064
:104AF0000E94901F2F9A0E94951F84788438D9F3C2
:104B0000D5CF0E948E1F88EC90E00E94901F2E98B7
:104B100082E090E00E945B30882329F060E082E030
:104B200090E00E94633084EF91E00E94901F2E9AE3
:104B30000E94951F84718431D9F3BDCF0E948E1FCE
:104B400082E090E00E945B30882319F00E94C81F29
:104B500002C00E94C31F2E98EEEE4E2E55245A948A
:104B600008E010E00E94951F86FF04C02E9A2F9A3D
:104B70002D9A92C02CEF42162FEF520619F42E9A5E
:104B80002F9806C048E14416510411F42F9A2D982D
:104B90000E94532350EF45165FEF55068CF40E9498
:104BA00060238BE190E00E94901F60EF46166FEF4C
:104BB000560609F059C08AEF90E00E94901F54C039
:104BC000920157FE04C02227332724193509277084
:104BD0003327C20157FC079673E0959587957A9520
:104BE000E1F757FE05C00197F801E21BF30B9F01A7
:104BF0007C01F694FE2CEE24F794E79440E050E01C
:104C00004801821A930AB70160587F4F5B018F3FBA
:104C10007FEF970744F40196485A5F4F7501403B78
:104C2000510589F7BCCFD701A65DBD4F60E070E0AC
:104C30008F3FEFEF9E0709F4ACC7FB01E40FF51FB0
:104C4000E455FF4FE4916D01CA18DB08CE0CDF1C60
:104C5000F0E01F01022E01C0220C0A94EAF7F601CF
:104C600070802728208295C7FFEF4F1A5F0A29E13D
:104C70004216510409F076CF8CEB92E00E94901F0F
:104C80000E948E1FE0910106F09102060190F081D2
:104C9000E02D81E096E0099582E390E00E94901F6C
:104CA0000E94951F8111F8CF80E1809308068091C2
:104CB00064008E7F8093640080917A00806480938A
:104CC0007A0080917A0086FDFCCF009178001091E7
:104CD00079000E94801C20E030E098011127002715
:104CE000600F711F821F931F61157105810591056A
:104CF00011F00E94523080916400816080936400C2
:104D00000E94602385E00E94171F8DE00E94171FFC
:104D10000E94532310921606109215061092140644
:104D2000109213064CE2242E3324339430E7D32E12
:104D30002FB7F8948091570190915801A091590193
:104D4000B0915A012FBF40910D0650910E0660910F
:104D50000F067091100620911106222341F0209138
:104D60000906821B80931206109211060AC7841747
:104D70009507A607B70738F4481B423008F401C767
:104D80000E94B21FFEC621E02093110680930906FF
:104D900090930A06A0930B06B0930C062091080688
:104DA000820F911DA11DB11D80930D0690930E06DB
:104DB000A0930F06B093100680910406909105060B
:104DC00001969093050680930406809106068093D1
:104DD00007060E94951F809306060E945323109297
:104DE0001606109215061092140610921306809162
:104DF0005C01823009F44BC130F4882359F08130D2
:104E000009F459C0BCC6833009F457C2843009F490
:104E10003DC6B5C6C12CEE24E39400E320E34BEB82
:104E200057E268E070E088E090E00E94C2218BE4E5
:104E300090E0909314068093130688E090E090939E
:104E400016068093150682EB97E20E94722387E58F
:104E500090E0909314068093130682E190E0909383
:104E60001606809315068BEA97E20E94722386E568
:104E700090E0909314068093130686E290E090935E
:104E800016068093150684EA97E20E94722384E452
:104E900090E0909314068093130681E390E0909342
:104EA0001606809315068AE997E20E94722381E034
:104EB0000E94AF2164C68093010196E490930001A3
:104EC00095E0909369019093680110926B011092A4
:104ED0006A0110926601109264018093020184EBD2
:104EE0008093670186E18093620189E68093600187
:104EF00088E18093610180935F01109265011092B7
:104F0000630110925E0110925D01C12CEE24E394C6
:104F100008E220E54AE056E263E070E088E190E0D4
:104F20000E94C22110916D01123028F480E40E9489
:104F30004823811149C610916D01112329F080E2A7
:104F40000E94482381114CC680916D0149E2849FE3
:104F5000C0011124C12CEE24E39400E12AE146EDC6
:104F600055E26EE270E00A960E94C2210EE026E150
:104F70004AEA55E26FE270E08DE090E00E94C221C3
:104F800026E14EE755E26FE270E085E390E00E9493
:104F9000C221E12C26E142E555E26FE270E08DE0AE
:104FA00090E00E94C22126E146E255E26FE270E005
:104FB00085E390E00E94C22180915B01882379F013
:104FC00026E14AEF54E26FE270E08EE590E00E9445
:104FD000C221EE24E39426E14EEC54E211C0C12C30
:104FE000E12C0EE026E142EA54E26FE270E08EE549
:104FF00090E00E94C221EE24E39426E146E754E2C9
:105000006FE270E08EE590E00E94C22188E00E948D
:105010004823882309F4B3C580916D01811108C02C
:1050200082E080935C0181E08093020110926D0127
:1050300080916D01813039F482E080935C0180932E
:10504000020110926D0180916D018230B9F480915E
:105050005B01882319F00E94C31F02C00E94C81F71
:1050600060915B0182E090E069830E945B3069811E
:10507000681721F082E090E00E94633044E650E03F
:1050800060E070E080E991E00E941E2178C5C12CAB
:10509000EE24E39400E12AE146ED55E262E070E09F
:1050A00080E690E00E94C22180910101813089F464
:1050B000E12C0EE026E142E555E263E070E082E695
:1050C00090E00E94C221EE24E39426E14AEA55E2F0
:1050D00011C0C12CE12C0EE026E146E255E263E06E
:1050E00070E082E690E00E94C221EE24E39426E183
:1050F0004EE755E263E070E082E690E00E94C22154
:1051000080E20E944823882321F080916D01811163
:1051100073C580E40E944823882329F080916D01A3
:10512000853008F477C580E80E944823882329F059
:1051300080916D01833008F07BC580E10E94482397
:10514000882329F080916D01833008F47FC5109287
:105150006C0162E070E07B836A836A807B80F2E0AE
:105160006F1A71088A809B802FEF821A920AA12CF5
:10517000B12C10916C01250172E0470E511CD19E9B
:10518000A00111244A525E4DC12CEE24E3940CE19F
:105190002CE16A817B81C2010E94C221F0906D01E5
:1051A0001F1106C001E020E240E2B301C5010DC0BD
:1051B00000E02CE14CE16A817B81C2010E949323D3
:1051C0002AE14AE1B401C50103960E9493231F5FBF
:1051D00010936C018EE1A80EB11C9AE5A916B104DA
:1051E00041F6EA81FB81B096FB83EA83E234F10564
:1051F00009F0B3CFF29C5001F39CB00C1124A5012F
:105200004253554EC12CE12C06E22EE166E170E0DE
:105210008EE590E00E94C221A5014C59544EEE2427
:10522000E3942EE166E170E08EE590E00E94C221F9
:1052300084E00E944823882369F081E080935C0128
:1052400010926D0144E650E060E070E082E890E08A
:105250000E941E2188E00E944823882309F48FC4FD
:1052600044E650E060E070E080E991E00E941E2199
:105270009091020180916D01913069F480936B01EE
:105280000E944D3026E030E040E050E00E94713056
:1052900060936A010EC090910101913041F48093B6
:1052A0006B0110926D0182E08093010168C48093CC
:1052B0006A0183E080935C0162C481E090E0909396
:1052C00014068093130610E080916901181768F4A2
:1052D000E091FD05F091FE050190F081E02D63E085
:1052E0008DEF95E009951F5FEFCF10E00AEF8091F9
:1052F00068011817D0F40103C001112486589F4F8C
:1053000090931406809313061092160610921506B9
:10531000E091FD05F091FE050190F081E02D63E044
:105320008DEF95E009951F5FE2CF28EEA22E25E0D4
:10533000B22E09EE15E0F12CF5018081F3E0FF15A6
:1053400010F492E001C093E0891BF5018083893C51
:10535000A8F00E944D302EE130E040E050E00E9485
:1053600071306F57F50160830E944D3028E230E0C4
:1053700040E050E00E947130F8016083F801408104
:1053800050E0F501608170E021E081E096E00E944C
:105390001120F394F2E0AF0EB11C0E5F1F4F2AE014
:1053A000F212CACF00E010E021E04AE250E0B8017A
:1053B00081E096E00E9411200F5F1F4F0038110519
:1053C00099F7809167018823D1F18C3371F048F40B
:1053D000813099F448EC50E060E070E084EF91E0B7
:1053E0000AC0883711F0843B41F444E650E060E0A5
:1053F00070E08CE291E00E941E218CE390E090939B
:1054000014068093130689E190E09093160680932A
:10541000150680916701893718F08EE491E007C086
:105420008D3318F080E591E002C082E591E00E94A2
:10543000F02380916701815080936701FDC180E175
:105440000E944823882349F080916601811105C09C
:1054500080916501882309F407C480E20E944823F3
:10546000882349F080916601811105C08091650112
:10547000882309F410C480910201823051F488E03D
:105480000E944823882379F180916401882389F060
:105490002AC0813041F50E944D3029E130E040E0E2
:1054A00050E00E9471306130710581059105D9F499
:1054B000EBCF80916301811116C081E0809364017C
:1054C000E0916A01F0E0EE0FFF1FED5EFE4F80817C
:1054D0008B5F8093630146E950E060E070E08CE20E
:1054E00091E00E941E2180910201823051F484E0FB
:1054F0000E944823882379F180916401882389F0F0
:105500002AC0813041F50E944D3024E130E040E076
:1055100050E00E9471306130710581059105D9F428
:10552000EBCF80916301811116C082E0809364010A
:10553000E0916A01F0E0EE0FFF1FED5EFE4F81810A
:10554000845F8093630146E950E060E070E082E8A8
:1055500090E00E941E2140916601423009F5809141
:105560006201825080936201209165012150209355
:105570006501E0916B01F0E0EE0FFF1FED5EFE4F65
:10558000818190E00C96821B910930916101059711
:1055900014F4345003C0253018F43C5F309361019B
:1055A00020916401223009F5809160018E5F809323
:1055B000600130916301315030936301E0916A01E1
:1055C000F0E0EE0FFF1FED5EFE4F818190E00C9644
:1055D000831B910950915F01059714F4545003C047
:1055E000353018F45C5F50935F01433031F58091A2
:1055F0006201815080936201309165013150309396
:105600006501E0916B01F0E0EE0FFF1FED5EFE4FD4
:10561000818190E00C96831B910905972CF4809171
:105620006101845080936101353038F410925E013D
:10563000809161018C5F80936101233031F580910D
:1056400060018F5F8093600130916301315030932E
:105650006301E0916A01F0E0EE0FFF1FED5EFE4F87
:10566000818190E00C96831B910905972CF4809121
:105670005F01845080935F01353038F410925D01F2
:1056800080915F018C5F80935F0180916201893C12
:1056900010F01092620180916001863218F486E267
:1056A0008093600180916101873018F484E08093D9
:1056B000610180915F01873018F484E080935F017D
:1056C000413029F4809162018E5F80936201213024
:1056D00029F480916001825080936001809165017E
:1056E000882319F08150809365018091630188239C
:1056F00019F08150809363018091650181111FC071
:10570000413069F410926601E0916B01F0E0EE0F18
:10571000FF1FED5EFE4F80818093650110C01092E7
:105720005E01109265011092660188E1809361012B
:1057300080916901811103C084E080935C018091B4
:10574000630181111FC0213069F410926401E0915E
:105750006A01F0E0EE0FFF1FED5EFE4F8081809347
:10576000630110C010925D011092630110926401F8
:1057700088E180935F0180916801811103C084E01A
:1057800080935C012091620130E0255E3F4F809163
:10579000600190E08497281739070CF43FC080918E
:1057A0006601813021F411E080915D01811110E0EA
:1057B00000916401013009F0B5C280915E01811150
:1057C000B1C248EC50E060E070E084EF91E00E94EC
:1057D0001E2100935E0180916901815080936901CF
:1057E00083E080936601E0916B01F0E0EE0FFF1F14
:1057F000ED5EFE4F8181845F80936501111162C26D
:1058000082E080936401E0916A01F0E0EE0FFF1FF7
:10581000ED5EFE4F81818A5E80936301809162011B
:10582000893518F089E5809362018091600187FFD6
:1058300003C08FE7809360018091660181111FC0D2
:1058400080916B01A0906101B12C60906201712C7C
:10585000829D4001839D900C1124A4014253554E1A
:10586000C12CE12C06E22EE1B501C3010E94C22148
:10587000A4014C59544EEE24E3942EE165C08130CE
:1058800009F520916B01A0906101B12C609062013B
:10589000712C8CE791E0289F4001299F900C1124E6
:1058A000A4014A515E4EC12CE12C07E226E2B5016B
:1058B000C3010E94C221A4014C555D4EEE24E39425
:1058C00026E242C08230F1F420916B01A090610188
:1058D000B12C60906201712C84E791E0289F400117
:1058E000299F900C1124A401425D564FC12CE12C3C
:1058F0000AE22FE1B501C3010E94C221A40148516F
:10590000564F1FC0833021F520916B01A09061019B
:10591000B12C60906201712C86E391E0289F4001D8
:10592000299F900C1124A40146515E4FC12CE12CFB
:1059300008E22FE1B501C3010E94C221A4014B5727
:105940005D4FEE24E3942FE1B501C3010E94C22113
:1059500080916401811123C080916A01A0905F0150
:10596000B12C60906001712C4EE1641A7108829D27
:105970004001839D900C1124A4014253554ECC2428
:10598000C394E12C06E22EE1B501C3010E94C221BD
:10599000A4014C59544EEE24E3942EE126C08130EC
:1059A00049F520916A01A0905F01B12C60906001DF
:1059B000712C56E2651A71088CE791E0289F40012E
:1059C000299F900C1124A4014A515E4ECC24C3940B
:1059D000E12C07E226E2B501C3010E94C221A40125
:1059E0004C555D4EEE24E39426E2B501C3010E94BE
:1059F000C221C5C0823011F520916A01A0905F01DB
:105A0000B12C60906001712C6FE1661A710884E717
:105A100091E0289F4001299F900C1124A401425D30
:105A2000564FCC24C394E12C0AE22FE1B501C30107
:105A30000E94C221A4014851564F24C0833009F06E
:105A40009EC020916A01A0905F01B12C609060011E
:105A5000712C7FE1671A710886E391E0289F40016D
:105A6000299F900C1124A40146515E4FCC24C3946D
:105A7000E12C08E22FE1B501C3010E94C221A4017B
:105A80004B575D4FEE24E3942FE1AFCF9091690126
:105A900080916801891738F5C12CEE24E39400E168
:105AA0002EE34EE651E06EE070E081E290E00E946D
:105AB000C2212AE146ED55E26DE170E083E390E01A
:105AC0000E94C221E12C0EE026E142E555E26EE1A2
:105AD00070E085E390E00E94C221EE24E39426E189
:105AE0004AEA55E228C0981768F5C12CEE24E394E1
:105AF00000E12EE34EE651E06EE070E081E290E0DE
:105B00000E94C2212AE146ED55E26DE170E083E397
:105B100090E00E94C221E12C0EE026E146E255E22F
:105B20006EE170E085E390E00E94C221EE24E394F0
:105B300026E14EE755E26EE170E085E390E00E94D9
:105B4000C22110C084E390E0909314068093130662
:105B500089E190E0909316068093150689E691E01E
:105B60000E94722380910001882321F0815080934C
:105B7000000105C080E00E94AF2110926D010E94DB
:105B8000602380E090E0892B09F4D2C80E940000D5
:105B9000CDC82115310581F0FB01E40FF51FE45557
:105BA000FF4FE491F0E0082C02C0F595E7950A94C8
:105BB000E2F7DC90ED29EC936F5F7F4F119668352B
:105BC000710509F035C827C81F5F10936D0144E6C1
:105BD00050E060E070E082E890E00E941E21ABC9D6
:105BE000115010936D0144E650E060E070E082E8EF
:105BF00090E00E941E21A8C944E650E060E070E0F9
:105C000082E890E00E941E2180916D018150809376
:105C10006D017FCA44E650E060E070E082E890E009
:105C20000E941E2180916D018F5F80936D017BCA60
:105C300044E650E060E070E082E890E00E941E21BF
:105C400080916D01835080936D0177CA44E650E0E6
:105C500060E070E082E890E00E941E2180916D017A
:105C60008D5F80936D0173CA81E080936601E0913E
:105C70006B01F0E0EE0FFF1FED5EFE4F80818B5F4A
:105C80008093650146E950E060E070E08CE291E0CD
:105C90000E941E21E2CB82E080936601E0916B01BD
:105CA000F0E0EE0FFF1FED5EFE4F8181845F809379
:105CB000650146E950E060E070E082E890E00E9413
:105CC0001E21D9CB11E048EC50E060E070E084EF99
:105CD00091E00E941E2181E080935D018091680126
:105CE00081508093680183E080936401E0916A01B0
:105CF000F0E0EE0FFF1FED5EFE4F8181845F809329
:105D0000630111118BCD82E080936601E0916B01FC
:105D1000F0E0EE0FFF1FED5EFE4F81818A5E809303
:105D200065017CCD112309F479CD10E0CCCFCF9261
:105D3000DF92EF92FF920F931F93CF93DF931F9207
:105D4000CDB7DEB7182F062FE42E862F880F8E5F73
:105D500099830E94EC1783E00E94EC17F12EC12E6C
:105D60009981D92E8C2D8F19801798F4F601E7FEB2
:105D700002C0849101C080810E94EC17182F80E03E
:105D80000E94EC178123FFEFCF1ADF0A8111EACFBF
:105D900001C081E00F90DF91CF911F910F91FF9093
:105DA000EF90DF90CF9008950F931F93CF93DF93E1
:105DB0008C0181E090E00E945B3080FF31C08AE07E
:105DC00090E00E945B309FEF980F9E3F48F522E3E2
:105DD00030E0D80157963C932E93569728E330E055
:105DE00059963C932E935897CBE0D0E0D801ED9193
:105DF000FC910190F081E02D682FC8010995CE013A
:105E00000E945B302196C131D10581F70E94602349
:105E100088EE93E0DF91CF911F910F910C94901F2A
:105E2000DF91CF911F910F91089504970C94D42E78
:105E30008F929F92AF92BF92CF92DF92EF92FF929A
:105E4000CF93DF93E6E9F5E01382128288EE93E0C8
:105E5000A0E0B0E084839583A683B7838CE291E0D1
:105E6000918380838FEF9FEF95878487EDEFF5E037
:105E7000138212821186128620E1238790878783FE
:105E8000108A118A128A138A148A8EE391E0918310
:105E900080838CE491E095838483178A168A118E1F
:105EA000108E81E0828F138E848F158E8CE599E1A0
:105EB0009093E7058093E6050E944D30C8EED5E04B
:105EC00020E8822E912CA12CB12CA50194010E94D6
:105ED000713068830E944D3032E2C32ED12CE12C08
:105EE000F12CA70196010E94713069830E944D3008
:105EF000A50194010E9471306A830E944D30A70170
:105F000096010E9471306B830E944D30A50194016F
:105F10000E9471306C830E944D30A70196010E944F
:105F200071306D830E944D30A50194010E94713043
:105F30006E830E944D30A70196010E9471306F83DD
:105F40000E944D30A50194010E94713068870E9423
:105F50004D30A70196010E94713069870E944D3033
:105F6000A50194010E9471306A870E944D30A701FB
:105F700096010E9471306B870E944D30A5019401FB
:105F80000E9471306C870E944D30A70196010E94DB
:105F900071306D870E944D30A50194010E947130CF
:105FA0006E870E944D30A70196010E9471306F8765
:105FB0000E944D30A50194010E947130688B0E94AF
:105FC0004D30A70196010E947130698B0E944D30BF
:105FD000A50194010E9471306A8B0E944D30A70187
:105FE00096010E9471306B8BDF91CF91FF90EF9003
:105FF000DF90CF90BF90AF909F908F9008958F9239
:106000009F92AF92BF92CF92DF92EF92FF92CF9387
:10601000DF93EC01688179818A819B81611571052B
:106020008105910521F464E279ED8BE597E02DE19E
:1060300033EF41E050E00E94713049015A019B0169
:10604000AC01A7EAB1E40E9490306B017C01ACEE98
:10605000B4EFA50194010E949E30DC01CB018C0DB0
:106060009D1DAE1DBF1DB7FF03C00197A109B0481C
:1060700088839983AA83BB83BC01CD019F77DF917D
:10608000CF91FF90EF90DF90CF90BF90AF909F9017
:106090008F9008950E94FF2F08958FE091E00E9455
:1060A000FF2F089560930F017093100180931101E9
:1060B000909312010895F999FECF92BD81BDF89A8F
:1060C000992780B50895262FF999FECF1FBA92BD62
:1060D00081BD20BD0FB6F894FA9AF99A0FBE0196C9
:1060E0000895052E97FB1EF400940E94883057FDFA
:1060F00007D00E94A33007FC03D04EF40C948830E4
:1061000050954095309521953F4F4F4F5F4F0895E3
:1061100090958095709561957F4F8F4F9F4F089513
:106120000E94C530A59F900DB49F900DA49F800D37
:10613000911D11240895B7FF0C9490300E94903067
:10614000821B930B0895A1E21A2EAA1BBB1BFD0113
:106150000DC0AA1FBB1FEE1FFF1FA217B307E40746
:10616000F50720F0A21BB30BE40BF50B661F771F9E
:10617000881F991F1A9469F760957095809590957E
:106180009B01AC01BD01CF010895A29FB001B39F57
:10619000C001A39F700D811D1124911DB29F700D30
:1061A000811D1124911D0895EE0FFF1F0590F4919C
:1061B000E02D099481E090E0F8940C94DF30F8949D
:0261C000FFCF0F
:1061C200460101FFFFFFFF00E100000000000001A7
:1061D200000000090305070A020705080406060372
:1061E2000100C18081000000000000007918DF1C5E
:1061F20098198F189A189C19BA19000000002F20BC
:106202004E1861196019D42EFCFF0000152F3300BF
:046212003200310025
:00000001FF
